:100000000C9436020C946E020C946E020C946E02E8
:100010000C946E020C946E020C946E020C946E02A0
:100020000C946E020C946E020C94611B0C94331CA5
:100030000C945E160C946E020C946E020C946E027C
:100040000C946E020C946E020C946E020C946E0270
:100050000C946E020C94E6160C946E020C946E02D4
:100060000C946E020C946E020C946E020C946E0250
:100070000C946E020C946E020C946E020C946E0240
:100080000C946E020C946E020C946E020C946E0230
:100090000C946E020C946E020C946E020C946E0220
:1000A0000C946E020C946E020C946E020D050D05FC
:1000B00039053905A105CC06CC06CC06BF05580686
:1000C00069066906A01CC71CBF1DC71CBF1D131DE8
:1000D000361DBF1D8D1D9C1D29001E001F00200008
:1000E00021002200230024002500260027002D00E7
:1000F0002E002A004A002B0014001A0008001500E8
:1001000017001C0018000C00120013002F00300014
:1001100031004B00390004001600070009000A00F6
:100120000B000D000E000F0033003400280000000B
:100130004E00E10000001D001B0006001900050034
:1001400011001000360037003800E50052004D0065
:10015000E000E300E2000000000000002C000000CE
:1001600000000000E6000151500051004F00350032
:100170003A003B003C003D003E003F004000410093
:1001800042004300440045004C0001000100010012
:1001900001000100010001000100010046004700CC
:1001A000480001000100010001000100AA00A900AF
:1001B000A800B000010001000100010001000100E1
:1001C0000100010000000100010000000100010029
:1001D0000100010001000100010001000100010017
:1001E0000100010001000100010001000000000009
:1001F00000000100000000000000010001000100FB
:1002000001000100010001000100010001000100E6
:1002100001000100010001000100010001000100D6
:1002200001000100010001000100010001000100C6
:1002300001000100010001000100010001000100B6
:1002400001000100010001000100010001000100A6
:100250000100010001000100010000000100010097
:100260000000010001000100010001000100010087
:100270000100010001000100010001000100010076
:10028000010000000000000001000000000000006C
:100290000100010001000100010001000100010056
:1002A0000100010001000100010001000100010046
:1002B0000100010001000100010001000100010036
:1002C0000100010001000100010001000100010026
:1002D0000100010001000100010001000100010016
:1002E0000100010001000100010001000100010006
:1002F00000000100010000000100010001000100F8
:1003000001000100010001000100010001000100E5
:1003100001000100010001000000000000000100D8
:1003200000000000000001000100010001000100C8
:100330002403770069006C00620061002E007400E5
:100340006500630068002000570054003600350047
:100350002D00460000001603770069006C00620063
:1003600061002E0074006500630068000000040353
:10037000090409023B00020100A0FA09040000017F
:10038000030101000921110100012240000705813C
:100390000308000109040100010300000009211104
:1003A000010001226D0007058203200001120100F7
:1003B000020000000882652D000100010200010515
:1003C000010980A101850319012AB700150126B78B
:1003D00000950175108100C0050C0901A10185047B
:1003E00019012AA002150126A002950175108100AD
:1003F000C005010906A1018506050719E029E715D1
:100400000025019508750181020507190029EF15DE
:1004100000250195F075018102050819012905954E
:100420000575019102950175039101C00501090649
:10043000A101050719E029E71500250195087501B7
:1004400081029501750881010507190029FF150032
:1004500026FF0095067508810005081901290595F4
:100460000575019102950175039101C011241FBE0C
:10047000CFEFDAE0DEBFCDBF04B603FE18C0809137
:10048000B0029091B102A091B202B091B302873054
:10049000904BA740B04B59F41092B0021092B102A9
:1004A0001092B2021092B302E0E0F8E3099511E075
:1004B000A0E0B1E0E4E9FCE302C005900D92A838A9
:1004C000B107D9F722E0A8E8B1E001C01D92A03B36
:1004D000B207E1F70E94BE120C94481E0C94000073
:1004E00081E0089581E008950C94720208950C94BF
:1004F00076021F93CF93DF9300D000D01F92CDB729
:10050000DEB749835A836B8330918B0189819A814D
:10051000311114C0662359F0222349F00E940509C5
:10052000182F682F89819A810E94AE0803C00E940B
:10053000D908182F69817A81812F04C00E9405098A
:1005400069817A810F900F900F900F900F90DF913B
:10055000CF911F910C942910FC01262F40815181CD
:100560006281738184810C94790281E00895CF9334
:10057000DF93EC0160E00E94AC02BE01DF91CF91FD
:100580000C9477020C946F110C946B1108950E94D7
:1005900058070E94C6022FEF84E39CE02150804060
:1005A0009040E1F700C000000C940C170F931F93CC
:1005B000CF93DF938C0161E00E94AC02EC01B801A3
:1005C0000E9474028823F1F1B801CE010E94B71491
:1005D0008823C1F1B801CE010E94CB12882391F18A
:1005E000B801CE010E941314882361F1F8018281C1
:1005F000882309F1CB358DE5D807C1F050F4C1153A
:10060000FCE5DF0781F0CF3DDC45A9F40E943C0EFC
:1006100019C0CC35EDE5DE0761F0CD35DD4559F487
:100620000E947F0D08C00E94C7020CC00E94880D66
:1006300002C00E948B0DC801DF91CF911F910F91D5
:100640000C94700280E0DF91CF911F910F9108957B
:100650000E9440160C9441030E9444030C944616D9
:1006600008950C94300381E008950C9433030895A9
:10067000CF93C82F0E9431038C2F0E943503CF9156
:10068000089580E00C9438030E9413150C943803ED
:100690000E94131590918A01891721F080938A0195
:1006A0000C9438030895CF93DF93CDB7DEB72B9723
:1006B0000FB6F894DEBF0FBECDBF4F835887698752
:1006C0007A878B8761110E94CB0C9E012F5F3F4F71
:1006D00086E0F90111928A95E9F785E0FE013796E7
:1006E000D90101900D928A95E1F789819A814C8117
:1006F0005D81452B31F09F3F31F491E08F3F19F43C
:1007000003C091E001C090E090FF09C049815A8187
:100710006B817C818D819E810E94EC0B05C0C9019B
:100720000E94B5028111F2CF2B960FB6F894DEBF6E
:100730000FBECDBFDF91CF910895FC0180819181E3
:100740000E9447090895CF93882309F49CC0C82FBD
:100750008238C1F40E94131581FD95C069E3809130
:100760000201909103010E94FB150E94ED0C2FEFF6
:1007700081EE94E0215080409040E1F700C00000FD
:1007800069E319C0833801F50E94131580FD7BC011
:1007900063E580910201909103010E94FB150E9484
:1007A000ED0C2FEF81EE94E0215080409040E1F776
:1007B00000C0000063E580910201909103010E9456
:1007C0000616CF910C94ED0C8438C1F40E941315D9
:1007D00082FD59C067E480910201909103010E945B
:1007E000FB150E94ED0C2FEF81EE94E0215080402C
:1007F0009040E1F700C0000067E4DDCF8CEF8C0F84
:10080000813AD0F46C2F80910201909103010E94F3
:100810007B15882349F06C2F809102019091030190
:100820000E9406160E94ED0C6C2F8091020190919F
:1008300003010E94FB15C5CF80E28C0F883048F47D
:10084000C77081E001C0880FCA95EAF70E94AE0C1C
:10085000B8CFEBE5EC0FE33040F4F0E0E15CFE4FA5
:10086000808190E0CF910C943915C85AC73158F463
:10087000EC2FF0E0EE0FFF1FEF5EFE4F80819181C5
:10088000CF910C944F15CF910895882309F45BC044
:10089000682F823879F40E94131581FF54C069E3F0
:1008A00080910201909103010E94FB150E94ED0CC2
:1008B00069E310C08338B1F40E94131580FF43C070
:1008C00063E580910201909103010E94FB150E9453
:1008D000ED0C63E580910201909103010E940616E0
:1008E0000C94ED0C843879F40E94131582FF2BC010
:1008F00067E480910201909103010E94FB150E9420
:10090000ED0C67E4E7CF8CEF860F813A18F380E2B5
:10091000860F883048F4677081E001C0880F6A95BF
:10092000EAF70E94B40CDCCF8BE5860F833020F40D
:1009300080E090E00C943915685A673120F480E02B
:1009400090E00C944F1508951F93CF93DF93182FC9
:10095000EB010E94A303209741F08FE99FE00197EC
:10096000F1F700C000002197F6CF812FDF91CF91E2
:100970001F910C944504893319F060E070E002C0C7
:1009800060E570E00C94A404882321F00E94AE0C72
:100990000C94ED0C0895882321F00E94B40C0C9463
:1009A000ED0C0895CF92DF92EF92FF920F931F9379
:1009B000CF93DF937C01D62FC72FFC0112810581D5
:1009C00002950F700E94A40C8823B9F01123A9F09E
:1009D0008C2F807F803421F080E28D0F883068F08A
:1009E00080918A0282FD09C082E00E944D0D0E9422
:1009F000A40C91E0D82ED92601C0D12CCC2EC294C3
:100A00008FE0C8228C2D90E08C30910508F0C4C195
:100A1000FC01EA5AFF4F0C94F31D8C2F807FCF709E
:100A2000882311F0C295C07F112399F0CC2309F4DB
:100A30009FC180E28D0F883010F0D11104C08C2F3F
:100A40000E94AE0C03C08C2F0E94BE0C0E94ED0CC5
:100A50008FC18D2F0E944504CC2309F49DC180E2F3
:100A60008D0F883038F1DD2329F18C2F0E94C40CC2
:100A700024C08C2F807FCF70803211F0C295C07F50
:100A8000DD2319F0D130A1F13DC080918A0282FFAF
:100A900017C0112349F0CC2329F08C2F0E94AE0CF3
:100AA0000E94ED0C80E065C180E00E944504CC23EB
:100AB00009F472C18C2F0E94B40C0E94ED0C6CC121
:100AC000112371F0002341F0013031F40E94CE0C6B
:100AD0008C2B0E94D60C60C10E94CE0C8C2B1DC0AA
:100AE000002319F0013009F457C10E94E30C25C01E
:100AF000112321F0063008F04FC10EC0053008F078
:100B00004BC11BC0112361F0002331F0F701858137
:100B100080FF2EC18F7085838C2F0E94C4043CC13E
:100B2000002359F0D93309F034C1FFEF07EE13E089
:100B3000F15000401040E1F72AC18C2F0E94CB04F5
:100B40002BC18C2F86958695837019F0813061F0CA
:100B500023C1112321F08D2F9C2F937002C080E0C0
:100B600090E00E94391520C1112321F08D2F9C2F78
:100B7000937002C080E090E00E944F1515C18C2F49
:100B8000837009F047C011110BC12D2F22952695B6
:100B90002770220F220F6D2F6F70862F90E0A0E03C
:100BA000B0E0022E04C0880F991FAA1FBB1F0A9431
:100BB000D2F7D4FF10C04FE050E060E070E004C016
:100BC000440F551F661F771F2A95D2F74095509501
:100BD0006095709503C040E050E0BA01C695C69597
:100BE000C3708A019B01082B192B2A2B3B2BC901AF
:100BF000B801C23049F058F4C13019F00E94C4075E
:100C0000CFC00E94B207CCC00E94D607C9C00E94C4
:100C1000B007C6C0112319F08C2F817001C08695D2
:100C2000882309F4BDC02D2F229526952770220F09
:100C3000220F6D2F6F70862F90E0A0E0B0E0022EA3
:100C400004C0880F991FAA1FBB1F0A94D2F7D4FFB4
:100C500010C04FE050E060E070E004C0440F551F4A
:100C6000661F771F2A95D2F740955095609570952D
:100C700003C040E050E0BA01C695C695C3708A0132
:100C80009B01082B192B2A2B3B2BC901B801C23021
:100C900049F058F4C13019F00E94890881C00E94BF
:100CA00077087EC00E949B087BC00E94EA0778C03C
:100CB000CF70112339F08C2F0E9410088D2F0E94C5
:100CC000C4046EC08D2F0E94CB048C2F0E9431086B
:100CD00067C0D23F21F128F4D03F41F0D13FC1F0AD
:100CE00043C0D33F19F1D43F79F03EC0112341F006
:100CF000053008F051C08C2F8F710E9456084CC0EF
:100D0000063008F049C0F7CF80918A0282FF18C0F0
:100D1000112339F08C2F8F710E9410083DC01123D0
:100D2000C9F38C2F8F710E94310836C0112329F02E
:100D30008C2F8F710E94FB072FC00E94F6072CC0DA
:100D4000112349F0CF718C2F0E94100863E08C2F83
:100D50000E94320D21C081E00E944D0D0230E0F072
:100D600082E00E944D0D18C0112331F0002391F252
:100D70008D2F0E94A30310C0002399F2D93349F4A8
:100D80001FEF27EE33E0115020403040E1F700C064
:100D900000008D2F0E94450488EF8C0D843020F4D4
:100DA0000E9413150E943803DD20C9F00E94A00C98
:100DB00080FD15C0F70112820E949A0C0E94100853
:100DC000C7010E9410070E949A0CDF91CF911F91DA
:100DD0000F91FF90EF90DF90CF900C943108DF914E
:100DE000CF911F910F91FF90EF90DF90CF900895DA
:100DF0000F931F93CF93DF93EC01688179818A81F0
:100E00000E9452098C010E94AD080E949E07B80101
:100E1000CE010E94D204DF91CF911F910F910895CE
:100E2000CF93DF93EC01988189812B813C81232B27
:100E300031F08F3F31F481E09F3F19F403C081E02E
:100E400001C080E080FD1DC0CE010E94D60281114C
:100E500010C00E94A40C8823A1F08A81882389F005
:100E600080918A0282FD0DC082E0DF91CF910C94C7
:100E70004D0DCE010E94F806CE01DF91CF910C946A
:100E8000B702DF91CF91089580E090E00E9439157C
:100E900080E090E00E944F150E94CB0C0C94ED0C6A
:100EA00080910201909103010E9411160C94440755
:100EB0000E94BB0C0C94500792959F70963079F06D
:100EC00010F4925001C09A50923068F4803F69F05B
:100ED00018F4883E40F409C0843F29F406C0883ED7
:100EE00020F0813F11F080E0089581E00895FC0139
:100EF000808191810E9447090E945C070895CF93E9
:100F0000DF9300D000D01F92CDB7DEB70F900F90C7
:100F10000F900F900F90DF91CF910895CF93DF93B3
:100F200000D000D000D0CDB7DEB726960FB6F8942B
:100F3000DEBF0FBECDBFDF91CF9108950895089514
:100F40000C949F070C94A0070E94A2076093C20113
:100F50007093C3018093C4019093C5010C9444071E
:100F60000C94A4070F931F930091C2011091C30129
:100F70002091C4013091C501602B712B822B932BE2
:100F80001F910F910C94A4070F931F930091C2011E
:100F90001091C3012091C4013091C50160237123D8
:100FA000822393231F910F910C94A4070F931F93F7
:100FB0000091C2011091C3012091C4013091C5017B
:100FC00060277127822793271F910F910C94A40704
:100FD0000C949F070E94E8076093BE017093BF01C5
:100FE0008093C0019093C1010C94440760E070E0CD
:100FF000CB010C94EA070F931F9341E050E060E0AF
:1010000070E08A019B0104C0000F111F221F331FD3
:101010008A95D2F7C901B8011F910F910C94EA0784
:101020000F931F9341E050E060E070E004C0440F74
:10103000551F661F771F8A95D2F78091BE01909148
:10104000BF01A091C001B091C1018A019B01082B91
:10105000192B2A2B3B2BC901B8011F910F910C941E
:10106000EA070F931F9341E050E060E070E004C096
:10107000440F551F661F771F8A95D2F740955095EC
:10108000609570958091BE019091BF01A091C001C3
:10109000B091C1018A019B01082319232A233B2314
:1010A000C901B8011F910F910C94EA070F931F9388
:1010B00041E050E060E070E004C0440F551F661F3F
:1010C000771F8A95D2F78091BE019091BF01A091C0
:1010D000C001B091C1018A019B01082719272A2765
:1010E0003B27C901B8011F910F910C94EA070F9398
:1010F0001F930091BE011091BF012091C00130915A
:10110000C101602B712B822B932B1F910F910C949B
:10111000EA070F931F930091BE011091BF01209128
:10112000C0013091C10160237123822393231F9159
:101130000F910C94EA070F931F930091BE01109139
:10114000BF012091C0013091C10160277127822722
:1011500093271F910F910C94EA0708952FE0929F17
:10116000800D1124E82FE695E695E695877051E00D
:1011700001C0550F8A95EAF785E0E89FF001112438
:10118000E457FE4F20E030E070E04081CB01022EBA
:1011900002C0969587950A94E2F78170819584271D
:1011A0008523842781932F5F3F4F2530310569F7D1
:1011B00008952FE0929F800D1124682F6695669503
:1011C0006695982F977085E0689FB001112440E0E4
:1011D00050E080E0FB01E40FF51FE457FE4F208153
:1011E00030E0092E02C0369527950A94E2F7217067
:1011F0003327042E01C0220F0A94EAF7822B4F5F97
:101200005F4F4530510531F70895BF92CF92DF927D
:10121000EF92FF920F931F93CF93DF938C01C090B7
:10122000BE01D090BF01E090C001F090C10180915B
:10123000C2019091C301A091C401B091C501C82A17
:10124000D92AEA2AFB2ACFE1D0E0D701C6010C2E29
:1012500004C0B695A795979587950A94D2F780FD17
:1012600004C0219790F7B12C07C0BC2EB8018C2F79
:101270000E943C100197A9F38B2DDF91CF911F9114
:101280000F91FF90EF90DF90CF90BF900895CF9394
:10129000DF93EC010E940509BE010E943C10DF9122
:1012A000CF9108951F93CF93DF93EB0190918B0122
:1012B000992321F0CB010E94470913C0882349F0EC
:1012C000CB010E940509182F682FCE010E94AE089D
:1012D00004C0CB010E94D908182FBE01812F0E94A3
:1012E0003C10DF91CF911F9108951F93CF93DF930F
:1012F000C091C60116E08091C701C81799F0D0E0EF
:101300001C9FF0011D9FF00D1124E853FE4F4081FA
:10131000518162817381848195810E948E0721961B
:10132000C770E9CFDF91CF911F9108954091F801E7
:101330005091F9016091FA017091FB018091FC01DB
:101340009091FD010C948E07EF92FF920F931F93E3
:10135000CF93DF938091FD0182958F7009F065C076
:101360008091FA01882309F460C08091C601F09051
:10137000C7011091F8010091F9016091FB01709192
:10138000FC0191E01F3F09F090E0C0910001D09175
:101390000101292F96E0E92E8F1509F446C0611549
:1013A000710521F00F3F21F030E003C031E001C0B2
:1013B000322F90E030FD36C0E89EF001E99EF00D3E
:1013C0001124DF01A853BE4F11963C9111973013A1
:1013D00029C03C91311326C012963C9112973111CD
:1013E00021C013964D915C911497461B570B4C17D7
:1013F0005D07C0F48091FD018F7080618093FD01D5
:10140000E353FE4F80818F708061808388EF91E08D
:101410000E941007DF91CF911F910F91FF90EF90E5
:101420000C94750901968770B7CFDF91CF911F910A
:101430000F91FF90EF9008959F92AF92BF92CF923D
:10144000DF92EF92FF920F931F93CF93DF93CDB76D
:10145000DEB761970FB6F894DEBF0FBECDBF8C012B
:1014600085E0F801DE011D9601900D928A95E1F765
:10147000D8011296EC909091F801E091F901209139
:10148000FB013091FC012115310531F0EF3F31F4C2
:1014900081E09F3F19F403C081E001C080E0B82FD4
:1014A000B1709B2E80FD47C1D8014C9111965C9183
:1014B00011971396AD90BC90149788EFC82E81E0D9
:1014C000D82EF090FA01B501621B730B2091000138
:1014D00030910101FF2009F4D9C08091FD0162170C
:1014E000730708F095C0282F207F09F052C05E13C3
:1014F00013C0491311C0FE2CE1100EC08F70806123
:101500008093FD010E949609C6010E9410078091F8
:10151000FD01F80185834DC1AB2831F05F3F31F407
:1015200081E04F3F19F403C081E001C080E080FDFD
:1015300003C081E08E2502C080E090E0F82FF170BA
:10154000FF2E80FF1CC08091C6012091C70136E0AC
:10155000821709F40BC190E0389FF001399FF00D1C
:101560001124E853FE4F6181561306C06081461373
:1015700003C06281E61203C001968770E9CFFE2C9A
:10158000EE2009F416C18091FD0181608093FD0178
:1015900054C05E1306C0491304C0E11002C0F80134
:1015A00099C0C8010E947707882361F1EE2051F1AC
:1015B0002091FD01822F82958F7090E0029774F048
:1015C0008091F8019091F90198878F831986BB86E5
:1015D000AA862C87CE0107960E94100786E0F801A4
:1015E000A8EFB1E001900D928A95E1F70E94A4095D
:1015F0000E9496090AC05E1711F1C8010E94770780
:1016000081112CC0C8010E941007FF24F394D1C09F
:10161000282F207F81F77A2DB98AA88A6E2D898993
:101620000E947F0788EF91E00E94100786E0D601B4
:101630001D928A95E9F70E949609F12CBAC04913C8
:10164000DCCFE110DACFF8018583C8010E941007D2
:1016500086E0D6011D928A95E9F7ABC0EE2091F2A3
:101660002091FD01822F82958F7090E002970CF4FB
:10167000B5CF8091F8019091F9019A8389831B82FB
:10168000BD82AC822E83CE010196A6CF621773076E
:1016900008F044C0FE2CEE2009F4B4CF5E1330C035
:1016A00049132EC02091FD0120FD21C0822F82957B
:1016B0008F70482F50E041155105C9F0F80125837E
:1016C0004F30510541F08F5F982F9295907F822F78
:1016D0008F70892B8583C8010E94100786E0F8016E
:1016E000A8EFB1E001900D928A95E1F73CC086E049
:1016F000F801A8EFB1E001900D928A95E1F759C089
:10170000C8010E947707811169CF8091FD01816036
:101710008093FD01C8010E9410074BC07A2DB98A41
:10172000A88A6E2D89890E947F0786E0D6011D92C6
:101730008A95E9F718C0EE2009F464CFC8010E9429
:101740007707F82E882309F45DCF86E0F801A8EF2B
:10175000B1E001900D928A95E1F788EF91E00E9447
:101760009D030E94A4090E94960923C04D875E87AD
:101770008D859E850E944709292F22952F70223042
:1017800028F49F7039F0811105C00BC0243028F473
:101790009F7049F4805E883020F0C8010E941007D5
:1017A0009F2CF92C06C0D80115969C91907F91F73B
:1017B000F8CF8F2D61960FB6F894DEBF0FBECDBF68
:1017C000DF91CF911F910F91FF90EF90DF90CF901D
:1017D000BF90AF909F9008951F93CF93DF93CDB7A5
:1017E000DEB72C970FB6F894DEBF0FBECDBF4F8388
:1017F000588769877A878B879C87CE0107960E94D6
:101800001C0A8823D1F09F8188852A853B85232B5C
:1018100031F08F3F31F481E09F3F19F403C081E044
:1018200001C080E080FD47C04F81588569857A8579
:101830008B859C850E948E073EC086E0FE01379610
:10184000DE01119601900D928A95E1F7FF81E885FE
:101850006A857B856115710531F0EF3F31F481E0D8
:10186000FF3F19F403C081E001C080E080FD23C088
:101870002091C70130E0C9010196877099274091F6
:10188000C60150E084179507F1F1F983EA837D835F
:101890006C8396E0929FD001939FB00D1124A853C2
:1018A000BE4FFE01319601900D929A95E1F780931B
:1018B000C7010E94750916E08091C6019091C70189
:1018C000891771F1189FC001112488539E4F0E94FF
:1018D0001C0A882329F1E091C6011E9FF001112402
:1018E000E853FE4F408151816281738184819581EB
:1018F0000E948E078091C60190E00196877099271B
:101900008093C601D9CF0E9458071092C701109248
:10191000C601E8EFF1E086E0DF011D928A95E9F764
:101920002C960FB6F894DEBF0FBECDBFDF91CF91DE
:101930001F91089580911E0285958595859508953E
:1019400080911E028770089590911E02977081E029
:1019500009F480E008958091410208959091410238
:10196000892B8093410208958095909141028923AB
:10197000809341020895109241020895909140028F
:10198000892B80934002089580959091400289238D
:1019900080934002089510924002089580911F02A2
:1019A000089508950C94D10C0C94D20C90918A0255
:1019B00092FD08C090911F02981721F080931F029A
:1019C0000C94D40C089580911F02882329F0109262
:1019D0001F0280E00C94D40C0895CF93DF93E09124
:1019E0000201F0910301809141028083E0910201A4
:1019F000F0910301908180914002892B8083809136
:101A00001F02882381F0E0910201F091030190818F
:101A1000892B808380910201909103010E946515BA
:101A200081110E94E30CC0910201D091030140E2B8
:101A300050E06EEF71E0CE010E94F91D892B69F034
:101A400080E2FE01AEEFB1E001900D928A95E1F7E0
:101A5000CE01DF91CF910C941F15DF91CF910895A6
:101A60000C94D10C90918A0292FD10C098E0899F4D
:101A700090011124262B20931E020E9410088091B1
:101A80001E028595859585950C94300D0C94100853
:101A900010921E0280E00C94300D20911E02809561
:101AA000822380931E02982F977099F430E0482F7C
:101AB000082E000C550B2417350759F090918A0217
:101AC00092FD07C08595859585950E9431080C94F7
:101AD000480D089590918A0292FB222720F9281739
:101AE00069F080FB92F990938A028091890290912B
:101AF0008A020E94B80D82E00C944D0D08958091E9
:101B00008A0282FB882780F991E089270C946A0D6C
:101B100081E00C946A0D80E00C946A0D6FEF7FEF0A
:101B200080E090E00C94321E80E090E00E940E1E57
:101B300021E0893E9E4F09F020E0822F089582E047
:101B400090E00C94061E83E090E00C94061ECF9368
:101B500084E090E00E94061EC82F82E290E00E947E
:101B6000061E2C2F30E0A901582BCA01CF910895F1
:101B7000CF93C92F682F84E090E00E94141E6C2F31
:101B800082E290E0CF910C94141EAB01BC018FE077
:101B900090E00C94261EAB01BC0183E190E00C9414
:101BA000261E60E070E0CB010C94CB0D60E070E08D
:101BB000CB010E94C50D0C94D10D69EE7EEF80E043
:101BC00090E00E94321E60E082E090E00E94141ECD
:101BD00060E083E090E00E94141E1092C201109217
:101BE000C3011092C4011092C50160E084E090E04E
:101BF0000E94141E60E082E290E00E94141E60E0E9
:101C000085E090E00E94141E60E086E090E00E9473
:101C1000141E6FEF87E090E00E94141E40E050E039
:101C2000BA0188E090E00E94261E60E08DE090E01E
:101C30000E94141E40E050E0BA0188E190E00E944A
:101C4000261E60E087E190E00E94141E40E050E014
:101C5000BA018CE190E00E94261E60E070E080E214
:101C600090E00E94321E40E050E0BA0188E190E02E
:101C70000E94261E0C94D60D0C94DD0D682F8EE06C
:101C800090E00C94141E0E94CB1660935002709347
:101C90005102809352029093530260934C027093CE
:101CA0004D0280934E0290934F02089585B780684D
:101CB00085BF85B7806885BF089581E008950C943D
:101CC0005D0E08950C94610E0C94610E0C94640EDC
:101CD0000C94610E0C94680E0C94610E0E94560ECA
:101CE00088E191E10E9409150E946C0E0C946A0E25
:101CF0000E94620E0C94610E0E9432110C94370304
:101D00000E94B6160E9417120E947C0E0C94660E5A
:101D10005F926F927F928F929F92AF92BF92CF927B
:101D2000DF92EF92FF920F931F93CF93DF93CDB784
:101D3000DEB72A970FB6F894DEBF0FBECDBF0E9464
:101D40002C12C82E81110E94430E32E4832E32E001
:101D5000932E00E010E0502E802F0E9456115C015F
:101D6000F401619071904F01682679266114710425
:101D7000B1F40F5F1F4F0530110569F78FEF8983AD
:101D80008A831B820E94BF168160782F9D838C837B
:101D900049815A816B818D810E9453033AC08091A1
:101DA000540281FD0E945F11D12CEE24E394F12CAA
:101DB000C3018E219F21892B29F10E945F0E882368
:101DC000A9F0DE825F82AE20BF2081E0AB2809F45B
:101DD00080E088870E94BF168160782F9A87898764
:101DE0004E815F8168858A850E945303000F111F11
:101DF000F801EE5BFD4F80819181E826F926F182A2
:101E0000E08207C0D394EE0CFF1CFFE0DF12D0CFBE
:101E1000B0CF81E0C11001C080E02A960FB6F894DF
:101E2000DEBF0FBECDBFDF91CF911F910F91FF900D
:101E3000EF90DF90CF90BF90AF909F908F907F906A
:101E40006F905F9008950E94880E0C944803CF9382
:101E5000DF930E944110EC01811522E59207E8F51D
:101E6000811531E5930708F0B6C0883E910528F545
:101E7000803E910508F0E9C0883A910570F4853AF2
:101E8000910508F07AC08130910509F473C008F417
:101E9000D9C0049708F0D9C0D5C08F3B910508F090
:101EA000D1C0C85AD0E0CC0FDD1FCE5BDE4F099009
:101EB000D881C02DCE019464C9C0811540E5940736
:101EC00008F069C0811550E4950708F060C09A9544
:101ED00081159F4108F4B9C0B5C0811536E5930757
:101EE00028F5811545E5940708F092C0811554E561
:101EF000950708F087C0AC0143705527282F269519
:101F00002695C115D34508F06CC081E090E002C071
:101F1000880F991F4A95E2F740E2249F900111240F
:101F2000EC01C22BD32BCE019C6890C081152AE511
:101F3000920780F4811539E5930708F072C0811586
:101F400048E5940708F47EC0D82FCC27CE01806FD7
:101F5000906A7CC090568115904208F073C08D2F16
:101F60008F710E94D510DD27D0628F71AE01582B82
:101F7000CA016CC081E090E069C0C55AD0E0C05988
:101F8000DE4F8881C82FD0E0CE0190645FC0DF7043
:101F9000CE01906A5BC074E0969587957A95E1F7DB
:101FA000282F23703C2F337081E090E002C0880F0F
:101FB000991F3A95E2F79C68AC01522B9A019C2F2D
:101FC0009F709695969550E2959FE0011124C90166
:101FD0008C2B9D2B3BC0D82FCC27CE01816F906AD4
:101FE00035C081E090E002C0880F991F4A95E2F762
:101FF00050E2259F90011124EC01C22BD32BCE017E
:102000009A6824C0D82FCC27CE01846F906A1EC056
:102010000E94D5108F7190E0D82FCC27CE0190620E
:1020200015C08F700E94D51094E0D695C7959A95EB
:10203000E1F7CF70D0E0DC2FCC27D0699E01282BB0
:10204000C90104C080E090E001C0CE01DF91CF91D2
:1020500008952BE4829FC0011124FC012FE0729FA0
:10206000E00DF11D1124E60FF11DEE0FFF1FE852E8
:10207000FF4F8591949108950E9429100E94270F87
:1020800008958238910569F1B0F48133910509F41E
:102090006DC048F48932910509F463C08A32910514
:1020A00009F469C008958533910509F455C0893351
:1020B0009105B9F00895833E910569F138F4803EA9
:1020C0009105B1F0823E910509F10895863E910592
:1020D000A9F1873E9105B9F1843E910509F064C0EC
:1020E00023C02091890220FD4FC021FD4DC00895DD
:1020F0008091890280FD44C080918A0280FF44C0A3
:102100008091890284FD42C083EE4DC08091890296
:1021100082FF38C0F5CF8091890282FD33C0809163
:102120008A0280FD31C0ECCF80918A0281FF32C0EB
:102130008091890284FD2AC087EE35C08091890292
:1021400083FF26C0F5CF8091890283FD21C0809155
:102150008A0281FD1FC0ECCF8091890285FD1CC0E1
:102160001DC08091890285FD19C016C08091890229
:1021700086FD16C017C08091890286FD13C010C06D
:1021800089E311C082EE0FC080EE0DC080E00BC06D
:1021900086EE09C084EE07C089E205C085E303C06E
:1021A0008AE201C081E390E008959091890292FF54
:1021B0000DC0282F2871283019F4877F846006C04D
:1021C000282F2471243011F48B7F886093FF0DC079
:1021D000282F2871283119F4877E846106C0282FA2
:1021E0002471243111F48B7E886120918A0220FFB2
:1021F0000DC0382F3871383019F4877F816006C0E0
:10220000382F3171313011F48E7F886021FF0DC07D
:10221000282F2871283119F4877E816106C0282F64
:102220002171213111F48E7E886194FD877E08959D
:1022300080E008950C948E0D0E942C128FE39CE98F
:102240000197F1F700C000000E942C1280E00E946C
:10225000561180FF04C00E941A110C940C170895A7
:102260000C941C110E94940D811102C00E943C0E1E
:102270000E949F0D809354020E94A70D90938A02A2
:10228000809389020E9430110E94A30D682F70E094
:1022900080E090E00E94B0076091BE017091BF01A4
:1022A0008091C0019091C1010C94E807E82FF0E003
:1022B000EE0FFF1FEB56FD4F808191810895089529
:1022C00080EA8A95F1F7089500C008950C94601192
:1022D00008950C9468110C9469110C9468110C9475
:1022E0006D11F894E82FE295EF70F0E031A1282FFE
:1022F0002F7081E090E001C0880F2A95EAF7982FAF
:102300009095932391A392A1892B82A37894089509
:102310000F931F93CF93DF93C2E8D1E089918F3F52
:1023200011F00E94711181E0C738D807B9F7C3E7EF
:10233000D1E002E811E089918F3F11F00E94711104
:102340000C171D07C1F7DF91CF911F910F910895D1
:10235000BF92CF92DF92EF92FF920F931F93CF9392
:10236000DF938C01C62FD0E0CE018E579E4F6C01BB
:10237000FC0190819F3F09F450C0B62EF894E92FDC
:10238000E295EF70F0E081A19F7021E030E001C0A4
:10239000220F9A95EAF7822B81A382A12095282308
:1023A00022A378940E946411E3E7F1E042E851E04F
:1023B00021E030E0E12CF12C61916F3F89F0A62FF4
:1023C000A295AF70B0E090968C9190E06F7002C0D3
:1023D000959587956A95E2F780FD02C0C90102C014
:1023E00080E090E0E82AF92A220F331F4E175F079A
:1023F00019F7F60180818F3F11F00E94711161E0A1
:10240000E114F10409F460E08B2D0E946611CC0FF9
:10241000DD1FC00FD11FF982E882DF91CF911F919C
:102420000F91FF90EF90DF90CF90BF9008950E94A2
:1024300088118AE0E5E9F2E0DF01982F1D929A9574
:10244000E9F7EBE8F2E0DF011D928A95E9F785E014
:102450000E9477120C94C202FF920F931F93CF93A6
:10246000DF93CDB7DEB72A970FB6F894DEBF0FBE65
:10247000CDBF8E010F5F1F4F8AE0F80111928A9540
:10248000E9F7F12C6F2DC8010E94A811F394F5E033
:10249000FF12F8CF4AE050E0B8018BE892E00E94CA
:1024A000F91DFF24F394009709F4F12C892B41F0D6
:1024B0008AE0F801ABE8B2E001900D928A95E1F76D
:1024C0002F2D45E065E972E08BE892E00E947812DA
:1024D0000E94C4028F2D2A960FB6F894DEBF0FBE5D
:1024E000CDBFDF91CF911F910F91FF900895089577
:1024F000FF920F931F93CF93DF93F82E092F162F80
:10250000D72FC42F222349F081E0809357020E94E5
:10251000BF169093560280935502809157028823EC
:10252000D9F080915502909156020E94D7160597D6
:1025300098F0EF2DF02FA12FBD2F80E090E04C2FD1
:1025400050E08417950734F4219131912D933D93F8
:102550000196F7CF10925702DF91CF911F910F9103
:10256000FF9008950E94B9180E94800E0C94C5181F
:102570000E94C9180E94230F0C94E3180E945D1654
:102580000E94A0180E946E0E0E94B2120E94B81201
:102590000E94780EFBCFCF93DF93EC01FB01828189
:1025A000882309F43CC1C430FDE5DF0760F4CB3F6C
:1025B0009CE5D90788F49E0122503C452431310521
:1025C00008F02EC109C0C236EDE5DE0729F0C63A93
:1025D000FDE5DF0709F024C10E94A70D90938A0250
:1025E00080938902C1318CE5D80709F4C6C008F090
:1025F00042C0C930ECE5DE0709F49BC000F5C530E8
:102600008CE5D80709F485C078F4C330ECE5DE0723
:1026100009F478C008F07AC0C230DC4509F0F5C092
:10262000809189028160EFC0C7309CE5D90709F429
:1026300078C008F07AC0809189028061E4C0CD3012
:10264000FCE5DF0709F487C058F4CB309CE5D907D7
:1026500009F479C008F07BC08091890288606FC05E
:10266000CF30FCE5DF0709F480C008F082C080911C
:102670008902877FC8C0CE3F9CE5D90709F471C0A5
:1026800000F5C531FCE5DF0709F485C068F4C33106
:102690009CE5D90709F475C008F095C00E94580759
:1026A000809189028F77AFC0CC3FFCE5DF07A9F1AD
:1026B00008F054C0CB3FDC4509F0A7C080918A02E6
:1026C00040C0C230EDE5DE0709F489C058F4C115F9
:1026D0008DE5D80709F45AC008F069C080918A02D4
:1026E00082602FC0C236EDE5DE0709F47CC0C63A31
:1026F000FDE5DF0709F481C0C330DD4509F085C081
:1027000080E06EC08091890282607DC080918902E4
:1027100016C080918902886076C080918A028260AA
:102720004FC08091890280626EC08091890280646E
:102730006AC00E94580780918902806864C08460E2
:1027400062C081603DC0809189028E7F5CC08091B3
:1027500089028D7F58C08091890216C080918A02BB
:1027600018C080918A028D7F2BC0809189028F7E54
:102770004AC0809189028F7D46C0809189028F7BFB
:1027800042C080918902877F8B7F3DC080918A0201
:102790008D7F8E7F15C08091890282FB222720F9D0
:1027A00091E0922790FB82F990FB83F92CC08091F5
:1027B0008A02982F909591708E7F892B90FB81F9DA
:1027C00080938A0222C00E9458078091890287FB69
:1027D000222720F991E0922790FB87F914C081E02D
:1027E0000E943E0E12C08091890284FB222720F9AC
:1027F00091E0922790FB84F906C080918902982F7E
:10280000909590FB80F98093890280918902909144
:102810008A020E94B80D0E94580780E001C081E042
:10282000DF91CF910895CF93DF9386319C4541F599
:10283000EB010E94AB0C982F8A812091020130910C
:102840000301882379F09A7A81E009F480E080938B
:102850005802911102C069E201C065E3C9010E94FA
:10286000FB150AC080915802811102C069E201C0C3
:1028700065E3C9010E9406160E94ED0C80E001C0CC
:1028800081E0DF91CF9108950F931F93CF93DF9352
:10289000C42FD22FFC0182818823C9F040935B02B0
:1028A0000E94BF1690935A028093590280E28C0FC7
:1028B000883008F057C0C77081E001C0880FCA9502
:1028C000EAF7DF91CF911F910F910C94C40480918E
:1028D0005B02481330C08091590290915A020E94C5
:1028E000D716883C910538F510E21D0FCD17B9F0C9
:1028F00080E28C0F883040F4C77081E001C0880FFF
:10290000CA95EAF70E94CB04183028F581E09D2F84
:10291000977001C0880F9A95EAF70E94C404802F2F
:102920000E94BB041830F0F4D77081E001C0880F1A
:10293000DA95EAF70AC080E28C0F883098F4C77005
:1029400081E001C0880FCA95EAF7DF91CF911F910E
:102950000F910C94CB04802FDF91CF911F910F9199
:102960000C94BB04DF91CF911F910F9108950F93A9
:102970009C01CB01243F4CE5340731F188F4293D1B
:10298000FCE53F07D9F02A3D4CE5340779F1283DB5
:102990003C45A9F506E221EE41EE68ED7CE52BC051
:1029A000263FFCE53F07E1F0A8F0273F3C4539F51D
:1029B00007E225EE46EE67EF7CE51DC007E225EE57
:1029C00045EE69ED7CE517C006E221EE40EE64EFCE
:1029D0007CE511C007E225EE44EE65EF7CE50BC017
:1029E00006E221EE42EE66EF7CE505C008E221E05A
:1029F00045EE6AED7CE50E94441480E008C0FC01CD
:102A00008281882319F010925B0201C081E00F914E
:102A100008959093890180938801089590936102AD
:102A2000809360020895E0916002F0916102309716
:102A300021F00190F081E02D099480E00895E0916B
:102A40006002F0916102309799F0209110012223E9
:102A500059F02091890227FF07C0DC012C911196C3
:102A60002C93119726E02C930280F381E02D09949A
:102A7000089520915E0230915F022817390771F0A6
:102A800090935F0280935E02E0916002F091610298
:102A9000309721F00680F781E02D09940895209168
:102AA0005C0230915D022817390771F090935D0246
:102AB00080935C02E0916002F0916102309721F016
:102AC0000084F185E02D09940895FC0132968091EF
:102AD0001001882331F08091890287FF02C09EE1B6
:102AE00001C096E080E0915028F021912223D9F393
:102AF0008F5FF9CF0895662351F1209110012223B1
:102B0000E9F02091890227FF19C0462F4695469586
:102B100046954E31E0F4677021E030E002C0220FAC
:102B2000331F6A95E2F7FC01E40FF11D828190E00A
:102B30002823392381E0232B69F409C0FC01329654
:102B400008962191621729F0E817F907D1F780E07C
:102B5000089581E008959C01FC0132969FEF80E08A
:102B60004191461789F09F3F19F4411101C0982FF8
:102B70008F5F8630A9F79F3F39F0F901E90FF11D0A
:102B800097FDFA956283089508959C012A5F3F4F4F
:102B9000FC014281461301C01282019682179307FD
:102BA000B9F70895262F2695269526952E3168F497
:102BB000FC01E20FF11D677021E030E001C0220F3F
:102BC0006A95EAF78281282B22830895262F26957D
:102BD000269526952E3170F4FC01E20FF11D6770E9
:102BE00021E030E001C0220F6A95EAF7209582814A
:102BF00028232283089520911001222329F0209177
:102C0000890227FD0C94D2150C94AB15209110016C
:102C1000222329F02091890227FD0C94E6150C94BB
:102C2000C51520911001FC013296222331F08091CC
:102C3000890287FF02C08EE101C086E0DF011D929C
:102C40008A95E9F7089508950C94231683E08093FC
:102C500062020C942416811102C081E001C082E05E
:102C6000809362020C9424160C942B1681E08093BE
:102C700062020C9424160C94361608950C943D169A
:102C80000C943E160C943D160C943D160C943D1677
:102C9000CF930E9444160E942C120E944216C0E05C
:102CA0008C2F0E945611892B29F4CF5FC530C1F7B4
:102CB00080E001C081E0CF91089508951F920F92A6
:102CC0000FB60F9211248F939F93AF93BF93809170
:102CD0006302811113C080919F029091A002A09184
:102CE000A102B091A2024196A11DB11D80939F0245
:102CF0009093A002A093A102B093A202BF91AF91C2
:102D00009F918F910F900FBE0F901F9018958091FB
:102D1000A702843031F10E9428031092630220E45C
:102D200088E190E00FB6F894A895809360000FBEFC
:102D30002093600083B7817F846083BF83B7816005
:102D400083BF7894889583B78E7F83BF0FB6F8943E
:102D5000A895809160008861809360001092600067
:102D60000FBE08950E9458070C942C0382E084BD86
:102D700093E095BD9AEF97BD80936E0008952FB7AD
:102D8000F89480919F029091A002A091A102B0912D
:102D9000A2022FBF08952FB7F89460919F027091FF
:102DA000A0028091A1029091A2022FBF08959C01E0
:102DB0004FB7F89480919F029091A002A091A10238
:102DC000B091A2024FBF821B930B089578941F927B
:102DD0000F920FB60F9211248F939F93AF93BF93CF
:102DE00080919F029091A002A091A102B091A202B5
:102DF0000196A11DB11D80939F029093A002A09304
:102E0000A102B093A202BF91AF919F918F910F90B9
:102E10000FBE0F901F90189581E08093E00080E234
:102E20008093D8001092C9008FE19EE40197F1F7DA
:102E300000C0000087E090EBDC018093B00290932B
:102E4000B102A093B202B093B3029CE088E10FB646
:102E5000F894A895809360000FBE90936000FFCF18
:102E60008091870208950895CF93DF9320911001F8
:102E7000222339F02091890227FF03C060E222E07B
:102E800002C068E021E02093E9002FEF3091E800D4
:102E9000215035FD06C035ED3A95F1F700002111BE
:102EA000F5CF2091E80025FF1DC0EC0180911001B5
:102EB000811105C040E050E068E070E003C070E0C0
:102EC00040E050E0CE010E9455198091E8008E77D5
:102ED0008093E80080E2FE01A7E6B2E001900D9247
:102EE0008A95E1F7DF91CF91089580936402709302
:102EF0006602609365028091A702843001F582E04A
:102F00008093E9008FEF9091E800815095FD06C015
:102F100095ED9A95F1F700008111F5CF8091E800C9
:102F200085FF0DC040E050E063E070E084E692E091
:102F30000E9455198091E8008E778093E8000895EB
:102F4000BC0184E00C947517BC0183E00C947517E8
:102F500008958091A602811109C00E94E61A0E947C
:102F6000431B8091E20084608093E20008951092F8
:102F7000A60208950C943B166091A30281E06111B2
:102F800001C080E00C9426169091A70281E0943055
:102F900009F080E06091A3020C942B1642E061ECF2
:102FA00081E00E945F1A42E261EC82E00E945F1AB7
:102FB0009091A70281E0943009F080E06091A30233
:102FC0000C9434168091A902833009F461C030F466
:102FD000813071F0823009F49AC008958A3009F482
:102FE00086C08B3009F46CC0893009F0A8C020C0BD
:102FF0008091A802813A09F0A2C08091E800877F01
:103000008093E8008091AC029091AD02892B21F46D
:1030100060E287E692E003C060E080E090E070E06C
:103020000E94A0198091E8008B778093E8000895B2
:103030008091A802813209F082C08091AC02909107
:10304000AD02029708F07BC08091E800877F8093F3
:10305000E8008091E80082FD05C08091A7028111FF
:10306000F8CF6DC02091F3008091F20090E0922B98
:10307000029731F48091F100813011F0863021F413
:103080008091F100809387028091E8008B7753C094
:103090008091A802813A09F052C08091AC029091CF
:1030A000AD02892B09F04BC08091E800877F8093A7
:1030B000E8008091E80080FFFCCF8091100136C0CD
:1030C0008091A8028132D9F58091AC029091AD0235
:1030D000892BA9F58091E800877F8093E8000E9402
:1030E000941A8091AA02809310010C945807809141
:1030F000A802813221F58091E800877F8093E80063
:103100000E94941A8091AB02809388020895809166
:10311000A802813AA1F48091E800877F8093E800BB
:103120008091E80080FFFCCF809188028093F100BD
:103130008091E8008E778093E8000C94941A0895AB
:1031400084B7877F84BF0FB6F894A89580916000FC
:10315000886180936000109260000FBE90E080E86C
:103160000FB6F89480936100909361000FBE0C94A9
:1031700036160E94E61A0E94431BE2EEF0E08081C0
:103180008460808378940C94D81D84E091E00C9442
:103190000E158091A7028530A9F48091A702853091
:1031A00079F40E9487168091A5028823B1F30E94CA
:1031B0004816882391F30E943F190E945807EDCFCB
:1031C0000C94B216089508950C94E618292F33270D
:1031D00023303105C9F060F42130310581F022300F
:1031E000310509F044C08BE390E022E733E043C0AF
:1031F00021323105E1F02232310549F138C082E156
:1032000090E02DEA33E037C099278130910549F0ED
:1032100028F0029761F5E0E3F3E005C0EEE6F3E0A5
:1032200002C0E6E5F3E0849190E09F0124C06115BF
:10323000710541F061307105D1F489E090E02DE92C
:1032400033E019C089E090E024E833E014C0611550
:10325000710541F06130710551F48DE690E02FEB7E
:1032600033E009C080E490E02CE234E004C080E068
:1032700090E020E030E0FA0131832083089580E17E
:1032800089BD82E189BD09B400FEFDCF8091D800DF
:103290008F7D8093D8008091E00082608093E00071
:1032A0008091E00081FDFCCF0895CF92DF92EF92F4
:1032B000FF920F931F93CF93DF93EC018B017A0161
:1032C0000E94B31A811133C0E114F10439F0F701FF
:1032D00080819181081B190BC80FD91FC12CD12CDB
:1032E0000115110519F18091E80085FD16C0809146
:1032F000E8008E778093E800E114F10449F0F701CB
:1033000080819181C80ED91ED182C08285E00FC014
:103310000E94B31A882321F30AC089918093F10097
:1033200001501109FFEFCF1ADF0ADACF80E0DF91F9
:10333000CF911F910F91FF90EF90DF90CF90089564
:103340002091AE023091AF022617370748F0611581
:10335000710539F42091E8002E772093E80001C030
:10336000B901FC0120E06115710579F18091A70296
:103370008823F1F18530F1F18091E80083FD3CC0B4
:103380008091E80082FD2EC08091E80080FFEBCFA5
:103390002091F3008091F20090E0922B611571056D
:1033A00051F08830910538F421912093F10061505B
:1033B00071090196F3CF21E0089709F020E0809190
:1033C000E8008E778093E800CECF2111CFCF0AC0DE
:1033D0008091A702882361F0853061F08091E80038
:1033E00083FD0AC08091E80082FFF2CF80E008955B
:1033F00082E0089583E0089581E008952091AE026F
:103400003091AF022617370748F06115710539F47E
:103410002091E8002E772093E80001C0B901FC015B
:1034200020E06115710591F18091A702882309F4CC
:1034300040C0853009F43FC08091E80083FD3DC065
:103440008091E80082FD2FC08091E80080FFE9CFE5
:103450002091F3008091F20090E0922B61157105AC
:1034600059F08830910540F424912093F100319671
:10347000615071090196F2CF21E0089709F020E030
:103480008091E8008E778093E800CBCF2111CCCFDC
:103490000AC08091A702882361F0853061F0809195
:1034A000E80083FD0AC08091E80082FFF2CF80E04F
:1034B000089582E0089583E0089581E00895982FAB
:1034C000973068F59093E900981739F07091EC0007
:1034D0002091ED005091F00003C0242F762F50E092
:1034E00021FD02C09F5FECCF3091EB003E7F309317
:1034F000EB003091ED003D7F3093ED003091EB001B
:1035000031603093EB007093EC002093ED0050930A
:10351000F0002091EE0027FDE5CF80E008958F7048
:103520008093E90081E008958091A80287FF11C08F
:103530008091E80082FD05C08091A7028111F8CF3B
:1035400011C08091E8008B770BC08091A70288237F
:1035500049F08091E80080FFF8CF8091E8008E77F5
:103560008093E80008952091E4003091E50095E60D
:103570004091EC00842F817040FF23C08091E800CF
:1035800080FD1DC08091A702882399F0853099F0B5
:103590008091EB0085FD11C04091E4005091E50061
:1035A0002417350729F3915011F09A01E1CF84E0F7
:1035B000089582E0089583E0089581E0089580E011
:1035C00008954091E80042FFDDCF08950E94541B0A
:1035D0000E945C1BE0EEF0E0808181608083E8ED7A
:1035E000F0E080818F77808319BCA7EDB0E08C91EB
:1035F0008E7F8C9380818F7E80831092A6020895A7
:103600000F931F93CF93DF930E94541B0E945C1B68
:10361000C8EDD0E088818F7788838881806888832F
:1036200088818F7D888319BC1092A7021092A30213
:103630001092A5021092A40200EE10E0F801808121
:103640008B7F808388818160888342E060E080E0B6
:103650000E945F1AE1EEF0E080818E7F8083E2EECF
:10366000F0E0808181608083808188608083F801C0
:1036700080818E7F8083888180618883DF91CF9174
:103680001F910F910895E8EDF0E080818F7E808397
:10369000E7EDF0E080818160808384E082BF81E09B
:1036A0008093A6020C94001BE8EDF0E080818E7FF1
:1036B00080831092E20008951092DA001092E100E7
:1036C00008951F920F920FB60F9211242F933F93DC
:1036D0004F935F936F937F938F939F93AF93BF931A
:1036E000EF93FF938091E10082FF0BC08091E20095
:1036F00082FF07C08091E1008B7F8093E1000E94F0
:10370000D71D8091DA0080FF1FC08091D80080FF14
:103710001BC08091DA008E7F8093DA008091D900FF
:1037200080FF0DC080E189BD82E189BD09B400FE42
:10373000FDCF81E08093A7020E94A91705C019BCA4
:103740001092A7020E94B7178091E10080FF19C074
:103750008091E20080FF15C08091E2008E7F80930F
:10376000E2008091E20080618093E2008091D800C5
:1037700080628093D80019BC85E08093A7020E94E4
:10378000BC178091E10084FF30C08091E20084FF8B
:103790002CC080E189BD82E189BD09B400FEFDCF66
:1037A0008091D8008F7D8093D8008091E1008F7E3A
:1037B0008093E1008091E2008F7E8093E20080910F
:1037C000E20081608093E2008091A302882311F0DF
:1037D00084E007C08091E30087FD02C081E001C062
:1037E00083E08093A7020E94C4178091E10083FFC9
:1037F00029C08091E20083FF25C08091E100877F8E
:103800008093E10082E08093A7021092A30280914E
:10381000E1008E7F8093E1008091E2008E7F8093B3
:10382000E2008091E20080618093E20042E060E08B
:1038300080E00E945F1A8091F00088608093F00021
:103840000E94BA17FF91EF91BF91AF919F918F9115
:103850007F916F915F914F913F912F910F900FBE8C
:103860000F901F9018951F920F920FB60F92112470
:103870002F933F934F935F936F937F938F939F9378
:10388000AF93BF93CF93DF93EF93FF93C091E90082
:10389000CF708091EC00D82FD17080FDD0E81092CD
:1038A000E9008091F000877F8093F00078940E9477
:1038B000771C1092E9008091F00088608093F000FE
:1038C000CD2BCF70C093E900FF91EF91DF91CF91A5
:1038D000BF91AF919F918F917F916F915F914F9128
:1038E0003F912F910F900FBE0F901F9018951F932F
:1038F000CF93DF93CDB7DEB7AA970FB6F894DEBFAC
:103900000FBECDBFE8EAF2E08091F100819322E0A2
:10391000E03BF207C9F70E94E2178091E80083FFBD
:103920002EC18091A8029091A902492F50E04A30FF
:10393000510508F024C1FA01EE59FF4F0C94F31D14
:10394000803821F0823809F01AC108C08091A402A1
:103950009091A502992389F082600FC08091AC02FA
:103960008F70873008F00BC18093E9008091EB00E5
:1039700085FB882780F91092E9009091E800977FF5
:103980009093E8008093F1001092F100D1C0282FAD
:103990002D7F09F0F4C0882319F0823061F0EFC068
:1039A0008091AA02813009F0EAC0933009F080E0EA
:1039B0008093A5022EC08091AA0281112AC0809115
:1039C000AC028F702FEF280F263008F0D8C08093FC
:1039D000E9002091EB0020FF1CC0933021F480917E
:1039E000EB00806214C09091EB0090619093EB002B
:1039F00021E030E0A90102C0440F551F8A95E2F78B
:103A00004093EA001092EA008091EB008860809376
:103A1000EB001092E9008091E800877F8093E80036
:103A20000E94941AACC08111AAC01091AA021F77FB
:103A30008091E3008078812B8093E3008091E800FF
:103A4000877F8093E8000E94941A8091E80080FFAD
:103A5000FCCF8091E30080688093E300111102C0E5
:103A600082E001C083E08093A70289C08058823041
:103A700008F085C08091AA029091AB028C3D53E082
:103A8000950779F583E08A838AE289834FB7F894B2
:103A9000DE01139620E03EE051E2E32FF0E0509388
:103AA0005700E49120FF03C0E295EF703F5FEF7095
:103AB0008E2F90E0EA3010F0C79601C0C0968D932B
:103AC0009D932F5F243149F74FBF8091E800877F96
:103AD0008093E8006AE270E0CE0101960E94A0198E
:103AE00016C06091AC027091AD02AE014F5F5F4FA6
:103AF0000E94E418BC01892B09F441C09091E800B0
:103B0000977F9093E80089819A810E94FE198091A5
:103B1000E8008B778093E80032C0803881F580918F
:103B2000E800877F8093E8008091A3028093F100F2
:103B30008091E8008E7772CF811121C08091AA0216
:103B40009091AB0299270297D4F48091E800877F87
:103B50008093E8008091AA028093A3020E94941AA5
:103B60008091A302811106C08091E30087FD02C00D
:103B700081E001C084E08093A7020E94CE1780916B
:103B8000E80083FF0AC08091E800877F8093E80007
:103B90008091EB0080628093EB00AA960FB6F894B8
:103BA000DEBF0FBECDBFDF91CF911F910895089565
:103BB000CF938091A7028823A1F0C091E900CF7034
:103BC0009091EC00892F817090FD80E8C82B1092B5
:103BD000E9008091E80083FD0E94771CCF70C093BC
:103BE000E900CF910895EE0FFF1F0590F491E02DAD
:103BF0000994FB01DC0104C08D910190801921F42E
:103C000041505040C8F7881B990B0895F999FECF91
:103C100092BD81BDF89A992780B50895A8E1B0E0DA
:103C200042E050E00C943A1E262FF999FECF92BD47
:103C300081BDF89A019700B4021639F01FBA20BD71
:103C40000FB6F894FA9AF99A0FBE08950396272FA3
:103C50000E94151E0E94141E252F0E94151E242F3F
:103C60000C94151E0196272F0E94151E0C94141EED
:103C7000DC01CB01FC01F999FECF06C0F2BDE1BD2C
:103C8000F89A319600B40D9241505040B8F708951B
:043C9000F894FFCFD6
:103C9400C800200230173417A817A417A017331729
:103CA40001E200E900EA00B500B600B700CD0083E8
:103CB40001CC008A019201940121022302240225ED
:103CC40002260227022A02B300B4006F00700081AA
:103CD4008283E200E900EA00B500B600B700CD0037
:103CE4008301CC008A01920194012102230224025F
:103CF4002502260227022A02B300B4006F007000D6
:103D0400818283F5953132339392676636353497E1
:083D14009694F0F1F4F6F700BB
:00000001FF
